:020000040000FA
:04000000DD303A288D
:08000800A000030EA100831209
:1000100081018B100B11210E8300A00E200E090010
:0C007400203084008001840A80300402E7
:10008000031C3C281230B000602183160C3085051B
:1000900087018312850187010730990000309A009B
:1000A000103083168E008312603083168F00831207
:1000B0000030831691009F008312C83083168100A0
:1000C000831231309000003083168C008312103080
:1000D0008B00831610309B001C141A088312BD007D
:1000E000142281018E018F010B118B100B108C01DA
:1000F0008B178D2031198F204221B30B8B280310D1
:1001000085190314B90DF030390203192B220F3071
:1001100039020319252235227928640008000800D5
:1001200031110130B7008B132030370783169B0045
:100130001C141A088312A4001030370783169B0082
:100140001C141A088312A3000030370783169B0083
:100150001C141A088312A2008B17321CB52822091E
:100160000339A200A309A409A50901303702031D20
:10017000BC283D143E14682102303702031DC328F9
:10018000BD143E147E2103303702031DCA283D15DD
:100190003E14942104303702031DD128BD153E14AE
:1001A000AA2101303702031DD8283D103E14C0217A
:1001B00002303702031DDF28BD103E14D521033065
:1001C0003702031DE6283D113E14EA2104303702B0
:1001D000031DED28BD113E14FF21EE28B70A05309E
:1001E00037020318080093280130B600B300B400AA
:1001F000B500B70085018701B1138D20B30B1A2913
:10020000031085190314B90DF03039020319382988
:10021000B41F8501B41F8701B40B1A293708B6082B
:100220000319B60003191829FF3085008700B603AB
:100230009630B400311DFD283111321C24292D09BE
:100240000339AD00AE09AF098B1320303707BB006F
:100250002F08BA004B2110303707BB002E08BA0018
:100260004B2100303707BB002D08BA004B218B17FC
:1002700085018701B70AB60105303702031CFD2846
:10028000142208003E1C08003E101030BB003D0840
:10029000BA004B2108008B133A0883161C159A00EC
:1002A00083123B0883169B0055309D00AA309D00A9
:1002B0009C1464009C1859291C1183128B17080088
:1002C000831610309B001C141A088312BD0008000E
:1002D0003D146430D5005D27E0006730D5005D2710
:1002E000E1006530D5005D27C4006630D5005D278C
:1002F000CC000130C800FF30C0000800BD146430DD
:10030000D5006727E2006730D5006727E300653036
:10031000D5006727C5006630D5006727CD000130BE
:10032000C900FF30C10008003D156430D5007127B9
:10033000E4006730D5007127E5006530D5007127EE
:10034000C6006630D5007127CE000130CA00FF30EC
:10035000C2000800BD156430D5007B27E600673079
:10036000D5007B27E7006530D5007B27C7006630C6
:10037000D5007B27CF000130CB00FF30C300080041
:10038000601A0512E01A8512601B0510E01B85102B
:1003900061188710E118071161190710E119871218
:1003A000611A0712E11A87110800621A0512E21A8F
:1003B0008512621B0510E21B851063188710E31875
:1003C000071163190710E3198712631A0712E31A5A
:1003D00087110800641A0512E41A8512641B0510BF
:1003E000E41B851065188710E518071165190710BB
:1003F000E5198712651A0712E51A87110800661AAF
:100400000512E61A8512661B0510E61B8510671893
:100410008710E718071167190710E7198712671A7D
:100420000712E71A871108003D186821601C3D106B
:10043000BD187E21621CBD103D199421641C3D1124
:10044000BD19AA21661CBD1108003D1808003D1405
:1004500068213E1408003D10C021BD10D5213D117A
:10046000EA21BD11FF213E140800D001D01B6821F4
:10047000501B7E21D01A9421501AAA210A300F0253
:10048000031C08008E018F013D1C612AC80B612AE4
:100490004C08C800C00A4408400203185D2A4008FE
:1004A000D5005D27D0004008D5006227D100600844
:1004B000E8006108E9002027612AC00160184F2A7E
:1004C0003D10BD1C7E2AC90B7E2A4D08C900C10AF9
:1004D0004508410203187A2A4108D5006727D00051
:1004E0004108D5006C27D1006208E8006308E900E4
:1004F00020277E2AC10162186C2ABD103D1D9B2A4F
:10050000CA0B9B2A4E08CA00C20A460842020318B8
:10051000972A4208D5007127D0004208D5007627D7
:10052000D1006408E8006508E90020279B2AC20181
:100530006418892A3D11BD1DB82ACB0BB82A4F0873
:10054000CB00C30A470843020318B42A4308D50066
:100550007B27D0004308D5008027D1006608E8003B
:100560006708E9002027B82AC3016618A62ABD112A
:02057000080081
:10060000003401340234033404340534063407342E
:10061000083409340A340B340C340D340E340F34DE
:10062000103411341234133414341534163417348E
:10063000183419341A341B341C341D341E341F343E
:1006400020342134223423342434253426342734EE
:10065000283429342A342B342C342D342E342F349E
:10066000303431343234333434343534363437344E
:10067000383439343A343B343C343D343E343F34FE
:1006800040344134423443344434453446344734AE
:10069000483449344A344B344C344D344E344F345E
:1006A000503451345234533454345534563457340E
:1006B000583459345A345B345C345D345E345F34BE
:1006C0006034613462346334F13464341E343F3452
:1006D000003400340034003400340034003400347A
:1006E000003400340034003400340034003400346A
:1006F000003400340034003400340034003400345A
:10070000003401340234033404340534063407342D
:10071000083409340A340B340C340D340E340F34DD
:10072000103411341234133414341534163417348D
:10073000183419341A341B341C341D341E341F343D
:1007400020342134223423342434253426342734ED
:10075000283429342A342B342C342D342E342F349D
:10076000303431343234333434343534363437344D
:10077000383439343A343B343C343D343E343F34FD
:1007800040344134423443344434453446344734AD
:10079000483449344A344B344C344D344E344F345D
:1007A000503451345234533454345534563457340D
:1007B000583459345A345B345C345D345E345F34BD
:1007C0006034613462346334003400340034003403
:1007D0000034003400340034003400340034003479
:1007E0000034003400340034003400340034003469
:1007F0000034003400340034003400340034003459
:10080000003401340234033404340534063407342C
:10081000083409340A340B340C340D340E340F34DC
:10082000103411341234133414341534163417348C
:10083000183419341A341B341C341D341E341F343C
:1008400020342134223423342434253426342734EC
:10085000283429342A342B342C342D342E342F349C
:10086000303431343234333434343534363437344C
:10087000383439343A343B343C343D343E343F34FC
:1008800040344134423443344434453446344734AC
:10089000483449344A344B344C344D344E344F345C
:1008A000503451345234533454345534563457340C
:1008B000583459345A345B345C345D345E345F34BC
:1008C0006034613462346334F13464341E343F3450
:1008D0000034003400340034003400340034003478
:1008E0000034003400340034003400340034003468
:1008F0000034003400340034003400340034003458
:10090000003401340234033404340534063407342B
:10091000083409340A340B340C340D340E340F34DB
:10092000103411341234133414341534163417348B
:10093000183419341A341B341C341D341E341F343B
:1009400020342134223423342434253426342734EB
:10095000283429342A342B342C342D342E342F349B
:10096000303431343234333434343534363437344B
:10097000383439343A343B343C343D343E343F34FB
:1009800040344134423443344434453446344734AB
:10099000483449344A344B344C344D344E344F345B
:1009A000503451345234533454345534563457340B
:1009B000583459345A345B345C345D345E345F34BB
:1009C0006034613462346334003400340034003401
:1009D0000034003400340034003400340034003477
:1009E0000034003400340034003400340034003467
:1009F0000034003400340034003400340034003457
:100A0000003401340234033404340534063407342A
:100A1000083409340A340B340C340D340E340F34DA
:100A2000103411341234133414341534163417348A
:100A3000183419341A341B341C341D341E341F343A
:100A400020342134223423342434253426342734EA
:100A5000283429342A342B342C342D342E342F349A
:100A6000303431343234333434343534363437344A
:100A7000383439343A343B343C343D343E343F34FA
:100A800040344134423443344434453446344734AA
:100A9000483449344A344B344C344D344E344F345A
:100AA000503451345234533454345534563457340A
:100AB000583459345A345B345C345D345E345F34BA
:100AC0006034613462346334F13464341E343F344E
:100AD0000034003400340034003400340034003476
:100AE0000034003400340034003400340034003466
:100AF0000034003400340034003400340034003456
:100B00000034013402340334043405340634073429
:100B1000083409340A340B340C340D340E340F34D9
:100B20001034113412341334143415341634173489
:100B3000183419341A341B341C341D341E341F3439
:100B400020342134223423342434253426342734E9
:100B5000283429342A342B342C342D342E342F3499
:100B60003034313432343334343435343634373449
:100B7000383439343A343B343C343D343E343F34F9
:100B800040344134423443344434453446344734A9
:100B9000483449344A344B344C344D344E344F3459
:100BA0005034513452345334543455345634573409
:100BB000583459345A345B345C345D345E345F34B9
:100BC00060346134623463340034003400340034FF
:100BD0000034003400340034003400340034003475
:100BE0000034003400340034003400340034003465
:100BF0000034003400340034003400340034003455
:100C00000034013402340334043405340634073428
:100C1000083409340A340B340C340D340E340F34D8
:100C20001034113412341334143415341634173488
:100C3000183419341A341B341C341D341E341F3438
:100C400020342134223423342434253426342734E8
:100C5000283429342A342B342C342D342E342F3498
:100C60003034313432343334343435343634373448
:100C7000383439343A343B343C343D343E343F34F8
:100C800040344134423443344434453446344734A8
:100C9000483449344A344B344C344D344E344F3458
:100CA0005034513452345334543455345634573408
:100CB000583459345A345B345C345D345E345F34B8
:100CC0006034613462346334F13464341E343F344C
:100CD0000034003400340034003400340034003474
:100CE0000034003400340034003400340034003464
:100CF0000034003400340034003400340034003454
:100D00000034013402340334043405340634073427
:100D1000083409340A340B340C340D340E340F34D7
:100D20001034113412341334143415341634173487
:100D3000183419341A341B341C341D341E341F3437
:100D400020342134223423342434253426342734E7
:100D5000283429342A342B342C342D342E342F3497
:100D60003034313432343334343435343634373447
:100D7000383439343A343B343C343D343E343F34F7
:100D800040344134423443344434453446344734A7
:100D9000483449344A344B344C344D344E344F3457
:100DA0005034513452345334543455345634573407
:100DB000583459345A345B345C345D345E345F34B7
:100DC00060346134623463340034003400340034FD
:100DD0000034003400340034003400340034003473
:100DE0000034003400340034003400340034003463
:100DF0000034003400340034003400340034003453
:100E4000681E262F501C051250180516E81E2C2F60
:100E5000D01C8512D0188516681F322F501D051022
:100E600050190514E81F382FD01D8510D01985148E
:100E7000691C3E2F511C871051188714E91C442F00
:100E8000D11C0711D1180715691D4A2F511D0710D4
:100E900051190714E91D502FD11D8712D11987163A
:100EA000691E562F511E0712511A0716E91E5C2F94
:100EB000D11E8711D11A8715080003308A00D51377
:100EC0005508820003308A00D51755088200043087
:100ED0008A00D5135508820004308A00D5175508BA
:100EE000820005308A00D5135508820005308A003B
:100EF000D5175508820006308A00D51355088200A0
:0A0F000006308A00D517550882005C
:084000000F000300050003009E
:02400E00CC33B1
:10420000FF00FF00FF00FF00FF00FF00FF00FF00B6
:10421000FF00FF00FF00FF00FF00FF00FF00FF00A6
:104220000100FF00FF00FF00FF00FF00FF00FF0094
:10423000FF00FF00FF00FF00FF00FF00FF00FF0086
:104240001000FF00FF00FF00FF00FF00FF00FF0065
:10425000FF00FF00FF00FF00FF00FF00FF00050060
:10426000FF00FF00FF00FF00FF00FF00FF00FF0056
:10427000FF00FF00FF00FF00FF00FF00FF00FF0046
:10428000FF00FF00FF00FF00FF00FF00FF00FF0036
:10429000FF00FF00FF00FF00FF00FF00FF00FF0026
:1042A000FF00FF00FF00FF00FF00FF00FF00FF0016
:1042B000FF00FF00FF00FF00FF00FF00FF00FF0006
:1042C000FF00FF00FF00FF00FF00FF00FF00FF00F6
:1042D000FF00FF00FF00FF00FF00FF00FF00FF00E6
:1042E000FF00FF00FF00FF00FF00FF00FF00FF00D6
:1042F000FF00FF00FF00FF00FF00FF00FF000000C5
:00000001FF
